:020000040000FA
:1000000007309F0083169F01003086008500831211
:100010003830792001307920033079200F30792071
:10002000803079200430A500263084003E308520C1
:100030008316F030860081138312EF30AA00860009
:100040000430A000AA0C2A088600912006080F3868
:10005000A100A109031D2F28A00B22281D28060896
:100060000F38A400A409031D2F2883160030860032
:100070008312AA092A080F39AA002108F039AA0414
:100080002A0886001130A100A1032108A6202A0217
:10009000031D44282108860010302107A620860071
:1000A000AA00003083160030860083122A088000E0
:1000B000840A8520A50B1828203085200430A5004F
:1000C000293084002508C7208002031D732884037B
:1000D000A50B62282B3085202B3085200514A1200C
:1000E0000510A12078286E3085206F308520A12052
:1000F0000028860091200430850091200030850082
:10010000912004308500912008008600912006305F
:1001100085009120023085009120063085009120D5
:1001200008003230A300A200A20B9428A30B93284E
:100130000800FA30A300A200A20B9C28A30B9B2866
:1001400008009920992099209920080082071134ED
:1001500012341434183421342234243428344134F1
:1001600042344434483481348234843488343034E2
:10017000313432343334343435343634373438343B
:1001800039344134423443344434453446348207AC
:0A0190002A3431343234333434346D
:02400E00293F48
:00000001FF
